:1018B0004856522D544553540001340000004368EB
:1018C000616E6E656C000100000000000000000009
:0918D0000000000000000000000F
:0819C500015E010310FF18B9D7
:10000E008F3C43A40C75A5FF7590FFD282D283E47A
:05001E00900000F0223B
:1017F1001513A813EFF6A813E6702D900000E0FF73
:101801007401C8EFC8088002C333D8FCF4F590EF27
:10181100B40803D38001C3B39282900000E0B409FD
:0B18210003D38001C3B39283051322A0
:050003008F327F002296
:10182C008B328A338934120B0EAB35AA36A9371298
:10183C000B54AB32AA33A934900001120B27AB35F1
:0D184C00AA36A937900001120B667F022218
:0100080022D5
:0D19B800245265763A20343931362024005F
:10085900E47880F61219A5C2B575E104E4F5E275EC
:10086900E34075A401F5A5F5A675A72075B16775CF
:10087900B208121989E4FF12196A43EF04E4F53A40
:10088900F53B7D01AF3B1218D9053BE53B700205ED
:100899003AC39401E53A940040E8E4F520C20AC25B
:1008A90008C20EC20DC20C7880F608F67885F618D3
:1008B900F6788AF6F53AF53B74A2253BF8E4F60595
:1008C9003BE53B7002053A6414453A70EBE4F53AAE
:1008D900F53B74B6253BF8E4F6053BE53B700205AC
:1008E9003A6408453A70EBE5EF20E10CE5EF54086E
:1008F900D394004003D38001C392037D08E4FF121F
:100909001924E47889F67882F6AB10AA11A912782D
:1009190082E6FF75F010A4F58285F083120B27FE9D
:10092900788926F6EE600578820680DDEFD394009B
:100939004030AB10AA11A91290000D120C75120BC0
:100949000EFF7455120B54120B0E64556002D20C33
:1009590074AA120B54120B0E64AA6002D20CEF1285
:100969000B54E5EF5402D3940040047F018002E464
:10097900FF120F858F39E53920E036C20974FF78F7
:100989008CF608F608F608F67E007F107D007B00DD
:100999007A007992120CCB753FFF7540187541B0FA
:1009A9007542007543107B007A0079921216C58052
:1009B90002D2099019BFE493FF3395E0FEEF24D0EA
:1009C900FFEE34FFFE7C007D64120B88AA06AB079C
:1009D9009019BEE493FF3395E0FEEF24D0FFEE3487
:1009E900FFFE7C037DE8120B88EF2BFBEE3AFA90B1
:1009F90019C0E493FF3395E0FEEF24D0FFEE34FFF6
:100A0900FE7C007D0A120B88EF2BFFEE3AFEA3E471
:100A190093FD3395E0FCED24D0FDEC34FFCD2F7828
:100A290091F6ED3E18F6E53930E103020AE5E4F501
:100A39003AF53BE53BC4F8540FC868FFE53AC4549E
:100A4900F048FEAB10AA11A9128F82F583120B2769
:100A59007003020ADCE92FF9EA3EFA900004120B4E
:100A69002720E264E4F538E538C3785E965059E505
:100A79003BC4F8540FC868FFE53AC454F048AB10BA
:100A8900AA11A9128F82F583120B27FF7E00C006D7
:100A9900C0077D00E53BC4F8540FC868FFE53AC4B8
:100AA90054F048FEE92FF9EA3EFA90000D120C7550
:100AB9007889E68538F0A429F9EA35F0FAD007D023
:100AC90006120CCB0538809F053BE53B7002053AC1
:100AD900020A3C7F0112000EC20B8007E4FF1200DC
:100AE9000ED20BE4F53AF53B7A007B967D03AF3BDA
:100AF900121403053BE53B7002053AC39401E53A3C
:040B0900940040E430
:010B0D0022C5
:0519FC00788AE6FF22DD
:03002300020E9337
:100E9300C0E0C0F0C083C082C0D075D000C000C025
:100EA30001C002C003C004C005C006C00730992EAC
:100EB300C2997885067985E77881667010F678851A
:010EC300F638
:080EC40075220A0000D522FB93
:040ECC00C2B580111A
:080ED0007522140000D522FB7D
:100ED8007885E624B6F8E6F599209803020F6A208B
:100EE8009A07200A04C2988075C29A7884E6062474
:100EF800A2F8A699C2987884E6FFB4011378A2E60E
:100F0800FE70057884F6805AEE54072402788BF632
:100F1800EFB4020E788BE6B4090878A3E6240379C7
:100F28008BF77884E6FFB4140476008035EFC37835
:100F38008B96402E7884E624FFFDE434FFFC7B008A
:100F48007A0079A21212657884E624A1F8E66F6027
:030F580002800B09
:080F5B007522140000D522FBF1
:100F630012002678847600D007D006D005D004D0AE
:100F730003D002D001D000D0D0D082D083D0F0D023
:020F8300E0325A
:10147C0078A3E675F010A4AB102512F9E51135F040
:10148C00FA90000D120C75788AE6FF18E68FF0A41E
:10149C002525F582E435F0F583120B27FF7B007AC6
:0314AC00007923A1
:1014AF008F328B338A348935EA494B6016120B0E13
:1014BF00FFE532FD7C001219D1AB33AA34A935EF09
:0314CF00120B54A9
:0814D2007536140000D536FB4D
:0E14DA008532997F011218593099FDC299226E
:1019000078B676787884E624A1F8E678B7F67F0290
:061910007881EFF6D2B56C
:081916007532140000D532FB0C
:06191E0078B6E6F59922FF
:10176800C9EFC9E964017028EDC39B4034785EE68F
:10177800FFEB2FFFE433FEEDC39FEE6480F8748027
:1017880098501ED20AC3ED9B788AF6788676012295
:10179800B90214ED6B700AD20A788AF67886760256
:0817A80022C20AE47886F62251
:1015BB00C9EFC9BAFF15BBFF12ED6B7002EC6A7075
:1015CB0049D20A788AF67886E9F622E96401702511
:1015DB00C3ED9BEC9A401C785EE62BFFE43AFEC30E
:1015EB00ED9FEC9E500DD20AC3ED9B788AF6788660
:1015FB007601228015B90218ED6B7002EC6A700A45
:10160B00D20A788AF67886760222C20AE47886F6BF
:01161B0022AC
:1000260078A2E6FF54F8F524EF120CA5006F09003C
:100036007B0A008D1000961100A61200BC1900D193
:100046001A00F32000F92801752902733302AB3731
:1000560002D13902EA4102F34902FC50034061022F
:1000660039700338980000036B78A3E6FD788DE6B7
:10007600FB7F01802578A3E6FC08E6FD788CE6FA8E
:1000860008E6FB7F018029D20A7886760302036B95
:1000960078A3E6FD788FE6FB7F0212176802036BF2
:1000A60078A3E6FC08E6FD788EE6FA08E6FB7F0212
:1000B6001215BB02036B78A3E6FD788DE6FB7F0184
:1000C600121768200A0302036B801978A3E6FC085E
:1000D600E6FD788CE6FA08E6FB7F011215BB200ADE
:1000E6000302036B78B676787F0102036875EF101A
:1000F60002036BC2ACE4F523D2B5FB7A0079237F09
:100106007F1214AF7B007A0079237F181214AF7B1D
:10011600007A0079237F051214AF7882E61214A8BC
:10012600788CE61214A8788DE61214A8788EE6125A
:1001360014A8788FE61214A87890E61214A878917D
:10014600E61214A8E4F52574922525F8E61214A8FB
:100156000525E525C3941040EE7B007A007900AFB3
:04016600231214AF9D
:08016A0075310A0000D531FBDC
:1001720002022678A3E6FFC3788296400302022D8C
:10018200EF75F010A42512F9E51135F085102EF562
:100192002F8930C2ACE4F523D2B5FB7A0079237FF4
:1001A2007F1214AF7B007A0079237F0D1214AFAB5C
:1001B2002EAA2FA930120B0E1214A8AB2EAA2FA909
:1001C200309000011214A5AB2EAA2FA93090000284
:1001D2001214A5AB2EAA2FA9309000031214A5ABBE
:1001E2002EAA2FA9309000041214A5E4F525AB2EF7
:1001F200E5302405F9E4352FFA7E00E92525F9EEEC
:100202003AFA120B0E1214A80525E525C3940840EC
:0C021200DD7B007A007900AF231214AFEE
:08021E0075310A0000D531FB27
:10022600C2B5D2AC02036B78B67678E408F67F02E4
:100236000203681219F27814120C5078B6767C789C
:1002460014E678B7F67815E678B8F67816E678B94B
:10025600F67817E678BAF67C007D057B007A007999
:10026600B612126578BBEFF67F0602036878A3E63E
:10027600FFB4010F08E6FD08E6788CCDF608EDF62A
:10028600020338EFB4020978A4E6788CF602033844
:1002960078A3E6B4030C08E6FF08E6788ECFF608E6
:1002A600EFF6020338E4F525E525C378A396501545
:1002B60074A42525F8E6FF74922525F8EFF60525A2
:1002C600E525B410E3E478A1F680677A007B327DF9
:1002D60001788AE6FF12140378A3E6FDE4FF1219FB
:1002E6002402036B78A3E624FF9202807878A3E6C3
:1002F60024FF9201806F788AE66005752702800BDD
:10030600200D05752703800375270178B6767908D1
:10031600A6277C007D027B007A0079B612126578EA
:10032600B8EFF67F03121910E52764017037D20E75
:100336008002D208788076F1802B7A007B327D01AC
:100346007F0012140378B6767978A3E678B7F67C40
:10035600007D027B007A0079B612126578B8EFF656
:100366007F03121910E52464A0600302055D78A2DC
:10037600E664A1600302045D79A3E7C37882964030
:1003860003020454AB10AA11A91278A3E6FF75F074
:1003960010A4F58285F083120B27F527EF75F01070
:1003A600A429F9EA35F0FA900004120B2730E2305E
:1003B60078A3E6FF1200038F2778B6767F08A62774
:1003C600E5272402FDE433FC7B007A0079B612129D
:1003D6006574B82527F8EFF6E5272403FF02055ACA
:1003E60078A3E6FF120003C2ACE4F523D2B5E527F5
:1003F600D39406402B7B007A0079237F7F1214AFBB
:100406007B007A007923AF271214AFE4F525E525A2
:10041600C39527500712147C052580F205278018FE
:10042600E52724781214A8E4F525E525C395275079
:100436000712147C052580F27B007A007900AF2331
:030446001214AFDE
:0804490075310A0000D531FBFA
:1004510002054E78B676787F0102055A78A2E664E5
:10046100A2600302055D7882E6FF78A3E6FEC39FE2
:10047100400302055408E6FDC39F4003020554EE04
:100481009D400302055418E6F525E4F52CF52DE50C
:1004910025D378A4965026AF25120003AB10AA11DC
:1004A100A91275F010E525A4F58285F083120B27BA
:1004B100252DF52DE4352CF52C052580D2C2ACE493
:1004C100F523D2B5FB7A0079237F7F1214AFC3E500
:1004D1002D9480E52C940050028007E52C44801275
:1004E10014A8AF2D1214A978A3E6F525E525D37834
:1004F100A4965046E4F526AB10AA11A91275F01086
:10050100E525A4F58285F083120B27FFE526C39F1D
:100511005024E52575F010A429F9EA35F0FA900088
:100521000D120C75788AE6FF18E68FF0A4252612C5
:10053100149E052680C1052580B27B007A007900D2
:05054100AF231214AF0E
:0805460075310A0000D531FBFC
:10054E00C2B5D2AC800978B676787F01121910E563
:10055E002464587047FA7B327D01788AE6FF1214C4
:10056E00037535007536007537B77B007A0079A3B1
:10057E0012182C8F27E527247878B6F6E527240164
:10058E00FDE433FC7B007A0079B612126574B72550
:10059E0027F8EFF6E5272402FF121910E5246480F0
:1005AE006009E524648860030207347886E6B401A6
:1005BE000F7A007B327D01788AE6FF121403801ACF
:1005CE00E4F525E525C3785E96500F7A007B327DE3
:1005DE0001AF25121403052580E978A2E65407F52C
:1005EE0027B4070A75260108E6F527088005E4F505
:1005FE002678A3E6F5281527E528C37882964003CA
:10060E00020722AB10AA11A91275F010E528A4F565
:10061E008285F083120B27FFE527D39F40028F2799
:10062E007886E6B40109788AE6F52BF52A8009E486
:10063E00F52A785EE614F52B788AA62A788AE6D310
:10064E00952B4003020716E4F525E525C3952740B3
:10065E000302070BE52875F010A4AB102512F9E57F
:10066E001135F0FA900004120B2730E20302070650
:10067E00900001120B2764387031E527D3940440A3
:10068E000BE526252524A4F8E6FD804E7884E6C3E6
:10069E009525FF74A02FF8E6FDE52875F010A4ABA4
:1006AE00102512F9E51135F0FA802FAB10AA11A919
:1006BE001275F010E528A4F58285F083120B27FF42
:1006CE00C37884E69F2525252624A1F8E6FDE52896
:1006DE0075F010A429F9EA35F0FA90000D120C7598
:1006EE00788AE6FF18E68FF0A4FFE5252FF582E461
:1006FE0035F0F583ED120B660525020658AF28126C
:10070E0017F1788A0602064A788AA62AE5246488B2
:10071E007014800FE528B4FF0D78A4E6F520E524CB
:10072E00B48803121900E52464A8600302085878FF
:10073E0086E6B4010F7A007B327D01788AE6FF12DD
:10074E001403801AE4F525E525C3785E96500F7ADA
:10075E00007B327D01AF25121403052580E978A3B5
:10076E00E630E711547FFE08E6FDEEF52CEDF52D93
:10077E00752603800B78A3E6752C00F52D752602E1
:10078E0074A22526F8E6FF74A32526F8E6F5298F30
:10079E0028E528D395294003020855E528C3788219
:1007AE00964003020850AB10AA11A91275F010E57D
:1007BE0028A4F58285F083120B27F5277886E6B4F8
:1007CE000109788AE6F52BF52A8009E4F52A785E88
:1007DE00E614F52B788AA62A788AE6D3952B5058FC
:1007EE00E4F525E525C395275044E52875F010A4BA
:1007FE00AB102512F9E51135F0FA900004120B2713
:10080E0020E227E526252524A4F8E6FD90000D120A
:10081E000C75788AE6FF18E68FF0A4FFE5252FF514
:10082E0082E435F0F583ED120B66052580B5AF2811
:10083E001217F1788A0680A0788AA62AE52725263F
:0A084E00F526052802079F12190085
:01085800227D
:107000007880E664F16003027541E4F53DF53E7871
:0470100081E6601A9B
:0870140075430A0000D543FB9F
:10701C00053EE53E7002053D64107004E53D6427B5
:10702C0070E1C2AF75FFDE75FFADE4F539F53820C0
:10703C009829E4F53DF53E20981DC3E53E9488E57E
:05704C003D94135012F9
:0870510075430A0000D543FB62
:10705900053EE53E70E4053D80E0B2B480D48599F3
:1070690038C298E538641A6003027120F53DF53E8F
:0E70790020981DC3E53E9488E53D9413501207
:0870870075430A0000D543FB2C
:10708F00053EE53E70E4053D80E030989F859939D7
:10709F00C298E4F53DF53E20981DC3E53E9488E582
:0570AF003D9413501296
:0870B40075430A0000D543FBFF
:1070BC00053EE53E70E4053D80E020980302703B00
:1070CC00859939C298E4F53DF53E20981DC3E53EFF
:0870DC009488E53D9413501265
:0870E40075430A0000D543FBCF
:1070EC00053EE53E70E4053D80E020980302703BD0
:0970FC00859939C298D2B5C299F8
:087105007543140000D543FBA3
:06710D007599783099FD30
:0871130075430A0000D543FB9F
:10711B00C2B5027533E5386450706EF53DF53E200F
:0D712B00981DC3E53E9488E53D9413501275
:0871380075430A0000D543FB7A
:10714000053EE53E70E4053D80E020980302703B7B
:09715000859939C298D2B5C299A3
:087159007543140000D543FB4F
:087161007599793099FDC2997E
:087169007543140000D543FB3F
:087171007599013099FDC299E6
:087179007543140000D543FB2F
:06718100E4F5993099FDD0
:0871870075430A0000D543FB2B
:0F718F00C2B5027533E5386401702FD2B5C299CD
:08719E007543140000D543FB0A
:0871A6007599783099FDC2993A
:0871AE007543140000D543FBFA
:0671B600E4F5993099FD9B
:0871BC0075430A0000D543FBF6
:1071C400C2B5027533E53864026003027273F53D9B
:1071D400F53E20981DC3E53E9488E53D9413501276
:0871E40075430A0000D543FBCE
:1071EC00053EE53E70E4053D80E020980302703BCF
:1071FC00859939C298E4F53AE53913B392B4E53977
:10720C0025E0FEC3E49400EE94705029E5397F002C
:10721C0025E0FEC39460501DE5B654F04408F5B665
:10722C00758F038E3F8F408540828E83E4F053B67A
:0C723C00F0F58F8003753AFFD2B5C299BF
:087248007543140000D543FB5F
:087250007599783099FDC2998F
:087258007543140000D543FB4F
:06726000853A993099FD0A
:0872660075430A0000D543FB4B
:10726E00C2B5027533E5386403600302739CF53DC5
:10727E00F53E20981DC3E53E9488E53D94135012CB
:08728E0075430A0000D543FB23
:10729600053EE53E70E4053D80E020980302703B24
:1072A600859939C298E4F53DF53E20981DC3E53E23
:0872B6009488E53D9413501289
:0872BE0075430A0000D543FBF3
:1072C600053EE53E70E4053D80E020980302703BF4
:1072D60085993BC298E5391392B4E53925E0FEC39A
:1072E600E49400EE9470400302703BE5397D00257E
:1072F600E0FCC39460400302703BE5B654F04408DA
:10730600F5B6758F01E53B75F020A42DFFE5F03C41
:10731600F53F8F40E4F53CE53CC394205043E4F54B
:107326003DF53E20981DC3E53E9488E53D941350F7
:017336001244
:0873370075430A0000D543FB79
:10733F00053EE53E70E4053D80E020980302703B7A
:10734F000540E540AE3F7002053F14F5828E83E5A0
:10735F0099F0C298053C80B653B6F0E4F58FD2B5DC
:02736F00C299C1
:087371007543140000D543FB35
:087379007599783099FDC29965
:087381007543140000D543FB25
:06738900E4F5993099FDC6
:08738F0075430A0000D543FB21
:10739700C2B5027533E53864046003027438F53DFD
:1073A700F53E20981DC3E53E9488E53D94135012A1
:0873B70075430A0000D543FBF9
:1073BF00053EE53E70E4053D80E020980302703BFA
:1073CF00859939C298E53925E0F541754200E4F514
:1073DF003AF53DF53E0542E542AE417002054114D6
:1073EF00F5828E83E493253AF53A053EE53E700229
:0E73FF00053D7004E53D640270DBD2B5C29915
:08740D007543140000D543FB98
:087415007599783099FDC299C8
:08741D007543140000D543FB88
:06742500853A993099FD43
:08742B0075430A0000D543FB84
:10743300C2B5027533E5386405600302752BF53D6B
:10744300F53E20981DC3E53E9488E53D9413501204
:0874530075430A0000D543FB5C
:10745B00053EE53E70E4053D80E020980302703B5D
:10746B00859939C298E4F53DF53E20981DC3E53E5C
:08747B009488E53D94135012C2
:0874830075430A0000D543FB2C
:10748B00053EE53E70E4053D80E020980302703B2D
:09749B0085993BC298D2B5C29953
:0874A4007543140000D543FB01
:0874AC0075997F3099FDC2992A
:0874B4007543140000D543FBF1
:1074BC007599203099FDE53925E0FCE53B75F02008
:1074CC00A42400FFE5F03CF5418F42E4F53AF53C8D
:0274DC00C29953
:0874DE007543140000D543FBC7
:1074E600854282854183E493F5993099FD0542E50D
:1074F60042AE417002054114F5828E83E493253A2B
:0B750600F53A053CE53CB420CDC299ED
:087511007543140000D543FB93
:06751900853A993099FD4E
:08751F0075430A0000D543FB8F
:10752700C2B58008E538B4060375EF10E53864077F
:0A753700600302703B7880F6D2AFCB
:017541002227
:1014E8007F0012185920090B7A007B327D017F009A
:1014F800121403300C0B7A007B1E7D017F0012143E
:1015080003300817300D147A007B327D01788AE6A3
:10151800FF121403C208121124D209200B0C300D3B
:1015280009788076F1121124D20B300E08300D059F
:10153800C20E127000200D121219E8E47B2C7A01F9
:0B154800F9F8C3120C335002D20D2240
:0B19DD001208591214E812000880F8EC
:100D8900005EBCE2613FDD83C29C7E20A3FD1F4162
:100D99009DC3217FFCA2401E5F01E3BD3E6082DC52
:100DA900237D9FC1421CFEA0E1BF5D0380DE3C6242
:100DB900BEE0025CDF81633D7C22C09E1D43A1FF32
:100DC9004618FAA427799BC584DA3866E5BB590722
:100DD900DB856739BAE406581947A5FB7826C49A12
:100DE900653BD987045AB8E6A7F91B45C6987A2402
:100DF900F8A6441A99C7257B3A6486D85B05E7B9F2
:100E09008CD2306EEDB3510F4E10F2AC2F7193CDE1
:100E1900114FADF3702ECC92D38D6F31B2EC0E50D1
:100E2900AFF1134DCE90722C6D33D18F0C52B0EEC1
:100E3900326C8ED0530DEFB1F0AE4C1291CF2D73B1
:100E4900CA947628ABF517490856B4EA6937D58BA1
:100E59005709EBB536688AD495CB2977F4AA481691
:100E6900E9B7550B88D6346A2B7597C94A14F6A881
:100E7900742AC896154BA9F7B6E80A54D7896B3571
:0A0E8900000060B0CBD8E5F3F700DD
:0319CD0001530AB9
:1012650015131513A813ECF608EDF615131513153C
:1012750013A813C6EBC608C6EAC608C6E9C6E51331
:0412850024FCF5133D
:10128900F80808E4F6A813F608F6E5132407F9A800
:1012990013E6FE08E6FFC3099719E76480F8EE64D0
:1012A90080985037E5132404F8CBE6CB08E6FA0812
:1012B900E6F98F828E83120B27A813080866FFE5CB
:1012C900132403F8EFF6E6900D8993A8130808F69E
:1012D900A8130806E61870B20680AFA8130808E636
:0112E900FF05
:0712EA00E5132409F51322AE
:0B19D100ED6F7818F6E6900D8993FF8B
:0119DC0022E8
:10192400EF701E7598D0E589540F4420F58953C88B
:10193400E1438E10ED900E8893F58DD28ED2ACC219
:03194400BCD2AF63
:01194700227D
:101717007856120C5C00000000785A120C5C00002E
:101727000000784E7664E47819F67819E6FFC394DA
:1017370001502DEF25E025E0244FF8E4F6EF25E0F2
:1017470025E02450F8E4F6EF25E025E02451F8E4FD
:10175700F6EF25E025E02452F8E4F678190680CA6A
:01176700225F
:10198900D2AFD2A9C2BBE589540F4401F589758E3E
:0C19990002758CECE4F58AD28C02171762
:0211C7001513FE
:1011C900A813E4F6A813E6FFC394014003021262D0
:1011D900EF25E025E02452F8E6FFD394004066A805
:1011E90013E625E025E02450F8E67059EF30E015C4
:1011F900A813E6FF25E025E02452F8E6D394014040
:10120900047D0080067D01A813E6FF1217B0A8131C
:10121900E6FF25E025E02452F8E6B401057D011238
:1012290017B0A813E6FF25E025E02452F816E6607A
:1012390014EF25E025E02451F8E6FEEF25E025E04E
:101249002450F8EEF6A813E625E025E02450F8E648
:09125900600116A813060211CD74
:031262000513224F
:03000B0002137D60
:10137D00C0E0C0F0C083C082C0D0E8C0E0E9C0E0EA
:10138D00EAC0E0EBC0E0ECC0E0EDC0E0EEC0E0EFA5
:10139D00C0E0758CEC7856120C44EF2401FFE43E4E
:1013AD00FEE43DFDE43CFC7856120C50784E16E6FA
:1013BD00701B785A120C44EF2401FFE43EFEE43D0D
:1013CD00FDE43CFC785A120C50784E76641211C72D
:1013DD00121948D0E0FFD0E0FED0E0FDD0E0FCD007
:1013ED00E0FBD0E0FAD0E0F9D0E0F8D0D0D082D058
:0613FD0083D0F0D0E032C5
:1018D9001513A813EDF61513A813EFF6A813E6FFD1
:1018E900C39401500D08E6FEEF25E025E0244FF8EA
:0718F900EEF60513051322B2
:1014030015131513A813EAF608EBF61513A813ED35
:10141300F61513A813EFF6A813E6FFC39401505271
:10142300EF25E025E02452F8E67047A813E6FB25F4
:10143300E025E02450F8E67039A81308E625E00417
:10144300FFA813E6FA25E025E02452F8EFF6A813E7
:101453000808E6FE08E6FF7C007D0A120B9AEA25DF
:10146300E025E02451F8EFF6EB25E025E02450F8E1
:09147300E4F6E5132404F513224C
:1017B0001513A813EDF61513A813EFF6A813E6FFFB
:1017C000C39401501CEF25E025E0244FF8E660119A
:1017D000A81308E670047F0180027F00A81308EFB9
:1017E000F6A813E6700608E624FF92B40513051365
:0117F00022D6
:0919E800C2AF7856120C44D2AFD4
:0119F10022D3
:0919F200C2AF785A120C44D2AFC6
:0119FB0022C9
:101859001513A813EFF6A813E670057854F608F6E1
:10186900300F167853E675F064A4FFC37855E69FE8
:0C18790018E695F0500375FFA50513223A
:10196A00D20FE47854F608F6EF78536003F6800253
:0F197A00760A75FF0775FFA543B28075EF092246
:1019A500C20FE47854F608F6785376FF75FFDE75B6
:0319B500FFAD2261
:10194800785506E618700106300F167853E675F0DC
:1019580064A4FFC37855E69F18E695F0500375FF19
:02196800A522B6
:041885008E088F0931
:10188900E4F50AF50BC3E50B9509E50A9508501629
:101899007FE87E0312161C7F01121859050BE50B10
:0618A90070E3050A80DF78
:0118AF002216
:04161C008E0C8F0D94
:10162000D3E50D94FAE50C9400500FEFD3940040ED
:1016300041007E0300DEFD1F80F1850C0E850D0F3D
:10164000D3E50F94FAE50E940040157FFA7E001260
:10165000161C7406250FF50F74FF350EF50E80E08D
:10166000D3E50D9400E50C94004007AF0FAE0E12C9
:02167000161C46
:011672002255
:10155300754800754900754A427B007A0079407DE1
:011563000285
:081564008B448A4589468D473E
:10156C007F01121859AB48AA49A94A120BD0240082
:10157C00FFE5F03460FE85444B85454C85464DE4D3
:10158C00FDEDC39547501BEF2DF582E43EF583E44A
:10159C0093AB4BAA4CA94D8D82758300120B660D33
:0F15AC0080DFAB48AA49A94AE48547F0020BFB50
:10106D00753A12753B3475420075430075443C7BEF
:07107D00007A00793A7D02C0
:081084008B3E8A3F89408D413B
:10108C007880E664F160030211231219A5C2AFE562
:10109C00B654F04408F5B6758F01AB42AA43A94487
:1010AC00120BD02400FFE5F034607819F608EFF647
:1010BC00AA3FA940781DA63E08C6EAC608C6E9C6DE
:1010CC00E4781BF6781BE6C395415032781DCBE6CD
:1010DC00CB080806E618CAE6CA70010614F9120B0A
:1010EC000E781CF6E6FF78190806E618CCE6CC70EC
:1010FC00010614F5828C83EFF0781B0680C6E4F5AC
:10110C008F53B6F0AB42AA43A9448541F0120BFBB6
:07111C00D2AFE4FF12196AD3
:0111230022A9
:101673007880E664F1704AC2AF1219A5E5B654F05A
:101683004408F5B6758F03781A7660087600E47817
:1016930019F6781AE6FE08E6F5828E83E4F07F01F8
:1016A300121859781BE426F618740236F61806E663
:1016B300C3940840DDE4F58F53B6F0D2AFFF12199F
:0116C3006ABC
:0116C4002203
:10112400121673E4F53CF53DF54275430075443CF5
:10113400FB7A00798C7D1612108412106DE4F53957
:10114400E539C3785E965073E4F538AB10AA11A95B
:101154001275F010E538A4F58285F083120B276030
:1011640056E53875F010A429F9EA35F0FA90000D27
:10117400120C757889E68539F0A429F9EA35F0FA74
:10118400EBC0E0EAC0E0E9C0E0AB10AA11A9127517
:10119400F010E538A4F58285F083120B27FD754223
:1011A4000075430075443CD0E0F9D0E0FAD0E0FB90
:1011B400121084053880940539808512106DE47806
:0211C40080F6B3
:0111C6002206
:020F85008F3C9F
:100F8700E4F542F543F53FF548754900754A42FBDC
:100F97007A00798C7D16121564121553E541643475
:100FA7007004E54064127003433F01E4F53EE53EFB
:100FB700C3785E964003021058E4F53DAB10AA11C2
:100FC700A91275F010E53DA4F58285F083120B2771
:100FD700607AE53C6054E53D75F010A429F9EA35DF
:100FE700F0FA90000D120C757889E6853EF0A42979
:100FF700F9EA35F0FAEBC0E0EAC0E0E9C0E0AB108F
:10100700AA11A91275F010E53DA4F58285F08312A7
:101017000B27FD754800754900754A42D0E0F9D0A5
:10102700E0FAD0E0FB121564801DAB10AA11A912DB
:1010370075F010E53DA4F58285F083120B27254353
:10104700F543E43542F542053D020FC3053E020F65
:10105700B5121553E54164347004E540641270031A
:05106700433F02AF3F12
:01106C002261
:030000000212F1F8
:0C12F100787FE4F6D8FD7581BD0213384B
:100B0E00BB010689828A83E0225002E722BBFE02E5
:090B1E00E32289828A83E4932218
:100B2700BB010CE58229F582E5833AF583E0225083
:100B370006E92582F8E622BBFE06E92582F8E222CD
:0D0B4700E58229F582E5833AF583E49322E7
:100B5400BB010689828A83F0225002F722BBFE0180
:020B6400F3227A
:100B6600F8BB010DE58229F582E5833AF583E8F0C5
:100B7600225006E92582C8F622BBFE05E92582C871
:020B8600F22259
:100B8800EF8DF0A4A8F0CF8CF0A428CE8DF0A42E81
:020B9800FE223B
:100B9A00C2D5EC30E709B2D5E4C39DFDE49CFCEE76
:100BAA0030E715B2D5E4C39FFFE49EFE120CF7C3EB
:100BBA00E49DFDE49CFC8003120CF730D507C3E4E6
:060BCA009FFFE49EFE22E5
:100BD000BB010A89828A83E0F5F0A3E022500687F0
:100BE000F009E71922BBFE07E3F5F009E3192289B2
:0B0BF000828A83E493F5F074019322E5
:100BFB00BB010789828A83020D4C500B09C5F02774
:100C0B00F7C5F01937F722BBFE0D09F8E325F0F312
:100C1B00C5F019E338F322F889828A83740193258E
:080C2B00F0C5F0F8E493382253
:100C3300EB9FF5F0EA9E42F0E99D42F0E89C45F017
:010C4300228E
:0C0C4400E6FC08E6FD08E6FE08E6FF22DC
:0C0C5000ECF608EDF608EEF608EFF622D0
:100C5C00D083D082E493F608740193F6087402935F
:090C6C00F608740393F674047396
:100C7500BB010DE58229F582E5833AF583020D6B0B
:100C85005007E92582F8020D62BBFE07E92582F8C7
:100C9500020D74E58229F582E5833AF583020D7D1F
:100CA500D083D082F8E4937012740193700DA3A3DE
:100CB50093F8740193F5828883E4737402936860F2
:060CC500EFA3A3A380DFF2
:1016C5008B3C8A3D893EE4F544F545E5431543AE3B
:1016D50042700215424E6033AB3FAA40A941120B3E
:1016E5000EFFAB3CAA3DA93E0545E545AC4470025D
:1016F500054414F5828C83EF120B66EF60CD7401FF
:101705002541F541E43540F54080C0AB3CAA3DA9F3
:021715003E2272
:100CCB00EF4E6012EF60010EEDBB010B89828A8340
:100CDB00F0A3DFFCDEFA2289F05007F709DFFCA94D
:0C0CEB00F022BBFEFCF309DFFCA9F022A4
:1012FD000219DDE493A3F8E493A34003F68001F211
:10130D0008DFF48029E493A3F85407240CC8C333F1
:10131D00C4540F4420C8834004F456800146F6DFC0
:10132D00E4800B01020408102040809019C5E47E72
:10133D00019360BCA3FF543F30E509541FFEE493B5
:10134D00A360010ECF54C025E060A840B8E493A37C
:10135D00FAE493A3F8E493A3C8C582C8CAC583CAA7
:10136D00F0A3C8C582C8CAC583CADFE9DEE780BE5F
:0119D0000016
:100CF700BC000BBE0029EF8DF084FFADF022E4CCE1
:100D0700F875F008EF2FFFEE33FEEC33FCEE9DECA9
:100D1700984005FCEE9DFE0FD5F0E9E4CEFD22EDEF
:100D2700F8F5F0EE8420D21CFEADF075F008EF2F39
:100D3700FFED33FD4007985006D5F0F222C398FD2A
:050D47000FD5F0EA22C7
:100D4C00C5F0F8A3E028F0C5F0F8E5821582700232
:060D5C001583E038F022CF
:090D6200E6FB08E6FA08E6F922B6
:090D6B00E0FBA3E0FAA3E0F92289
:090D7400E2FB08E2FA08E2F922B0
:0C0D7D00E493FB740193FA740293F922D2
:00000001FF
